:1000000019C033C032C031C030C02FC02EC02DC087
:100010002CC02BC02BC029C028C027C026C025C09B
:1000200024C023C022C021C020C01FC04CC01DC09E
:100030001CC01BC011241FBECFEFCDBFDFE3DEBF4E
:100040001FE3A0E0BFE3E4EBF5E002C005900D92F2
:10005000A230B107D9F72FE3A2E0BFE301C01D92A0
:10006000AF31B207E1F7E5D19EC2CACF1F920F921E
:100070000FB60F9211248F9380910F3F811103C00F
:1000800082E0809306048091133F811103C080E4D5
:10009000809306048091173F811103C088E080930C
:1000A000060480911B3F811103C084E08093060405
:1000B00080E180930B0A10920A0A8F910F900FBE75
:1000C0000F901F9018951F920F920FB60F92112448
:1000D0002F933F934F935F936F937F938F939F9350
:1000E000AF93BF93CF93DF93EF93FF93C09100083B
:1000F00080910D3F90910E3F8330910509F472C0BD
:1001000058F58130910509F445C0029709F461C0A2
:10011000C7FF0FC08C2F807F803F59F4C83F09F480
:10012000FCC008F0D2C0C03F09F475C1C73F09F454
:100130007BC1FF91EF91DF91CF91BF91AF919F91E3
:100140008F917F916F915F914F913F912F910F9080
:100150000FBE0F901F9018958530910509F472C05D
:1001600008F459C00697A1F680910A3F8A3209F433
:1001700094C008F06EC0893209F05FC0C7FD5DC051
:10018000E091093F84E0E89FF0011124E15FF04C29
:10019000C08353C0E0910C3FF0E0E455FA47808102
:1001A0008C1721F010920D3F10920E3F80910C3F62
:1001B0008F5F80930C3F80910C3F843009F0A8CF73
:1001C00082E090E080930D3F90930E3F10920C3FA1
:1001D0009FCF80910B3F8C1711F0CF3771F583E0E3
:1001E00090E0F0CFE0910C3FF0E0E655FA478081D7
:1001F0008C1721F010920D3F10920E3F80910C3F12
:100200008F5F80930C3F80910C3F823009F080CF4C
:1002100084E090E0D7CFC13429F068F487ED8C0FEB
:10022000823058F4C0930A3F85E090E080930D3F00
:1002300090930E3F6DCFCF37A9F310920D3F1092E0
:100240000E3F66CFC430C8F7C093093F86E090E008
:10025000EDCF813471F18F3781F7E091093F84E070
:10026000E89FF0011124E15FF04C60818091093F2B
:1002700090E0880F991F019650D1E091093F84E0EA
:10028000E89FF0011124E15FF04C61818091093F0A
:1002900090E0880F991F029616C0C7FDCECFE0915F
:1002A000093F84E0E89FF0011124E15FF04CC18335
:1002B000C4CF8FEF8C0F8E3708F0BFCFC0930B3FAA
:1002C0006C2F90E080E029D1B8CFCB3F01F1CC3F3B
:1002D00009F491C0CA3F09F02CCF1092200A109265
:1002E000210A90E080E0FC01EE0FFF1FEE0FFF1FE0
:1002F000E15FF04C128221812383019684309105C5
:1003000091F782E08093073F8EE48093060481E0BA
:100310008093083F1092063F0CCF8091083F8823BE
:1003200009F407CF8091073F811140C08091200AD6
:100330009091210A969587958093003F9093013F75
:100340008091003F9091013F8093280A9093290A61
:100350001092200A1092210A80E180930B0A809368
:100360000A0A30E020E0E901CC0FDD1FCC0FDD1FD1
:10037000FE01E15FF04C8381882319F08381815075
:100380008383FE01E15FF04C8381811109C080818C
:10039000811112C0F901E055FA478081809305046C
:1003A0002F5F3F4F24303105F1F6C3CE8091073FD8
:1003B00081508093073FC4CF6081828190E070E0DC
:1003C0006F5F7F4FC9D082838281882341F0428151
:1003D0008081869590E001964817190631F4F9015D
:1003E000E055FA47808180930704C15FD04C8A8131
:1003F0008F5F8A83D5CF1092083F8091063F8F5F31
:100400008093063F8091063F823009F092CE8EE4C1
:10041000809306048ECE10920C3F81E090E0809392
:100420000D3F90930E3F85CE10920D3F10920E3FE0
:1004300080CEF894C1E088ED84BFC093610090E065
:1004400080E063D080930B3F8F3F31F4C0930B3F2C
:1004500061E090E080E061D001E010E0F12CE12C5F
:10046000C80153D0E701CC0FDD1FCC0FDD1FC15FEA
:10047000D04C888368018FEFC81AD80AC60145D0CE
:10048000898388818F3F41F4188219826881C8016D
:1004900044D06981C60141D08FEFE81AF80A0E5F97
:1004A0001F4F84E0E816F104D9F68FE7809300042B
:1004B000109204041092010280911704877F8093A8
:1004C000170480E094E0809308089093090880E87E
:1004D000809305088093060883E0809307081092B4
:1004E000000A8FE08093050A8FEF9FEF8093260A22
:1004F0009093270A80E898E18093280A9093290A2C
:100500008DE08093000A7894FFCF03D080819927F3
:100510000895FC01E050FC4E0895262F0E948902A8
:100520000080021619F00E94990201970197089520
:10053000262FAF93BF93E0E0F0E1328131FDFDCF94
:10054000DC01A050BC4E2C932DE924BF23E0208376
:100550000196BF91AF91089597FB072E16F4009472
:1005600006D077FD08D00BD007FC05D03EF490955F
:1005700081959F4F0895709561957F4F0895AA1BAF
:10058000BB1B51E107C0AA1FBB1FA617B70710F07E
:10059000A61BB70B881F991F5A95A9F780959095B0
:0A05A000BC01CD010895F894FFCFCF
:0A05AA0020000020131A024008048C
:0205B4008018AD
:00000001FF
